:020000000528D1
:080008008D28850107309900E5
:1000100083169F013C3095003C30850017308100ED
:1000200083120530A400FF30A300A40B18281C285D
:100030007820A30B182813288E200B1828280B14BF
:10004000FF230B105B2083160030900083122B28B7
:100050000B1000305B200000851E4520051E4D2042
:10006000051D5620000000000000851478200000C7
:100070000000000000000000000000000000000080
:1000800000000000851078202C2883161008043EFC
:1000900090008312851E4A28080083161008043039
:1000A000100290008312051E5328080069200514D1
:1000B000051D5828080083169A006F309B001C15F8
:1000C00055309D00AA309D009C149C186528831211
:1000D0000800831610089A007F309B001C155530CD
:1000E0009D00AA309D009C149C187428831208005F
:1000F0000130A1007530A2000000A20B7C28A10BEA
:100100007A2800000000000000000000000000004D
:1001100000000000000000000800090083163C30C9
:100120009A00603011212D309A00613011212D305C
:100130009A006230112143309A0063301121483017
:100140009A006430112149309A00653011215030F5
:100150009A006630112120309A00673011214F300B
:100160009A006830112153309A00693011214330D0
:100170009A006A30112141309A006B3011214C30C5
:100180009A006C30112120309A006D3011212030FE
:100190009A006E30112100309A006F3011213C30EE
:1001A0009A00703011212D309A00713011212D30BC
:1001B0009A00723011214E309A007330112145306F
:1001C0009A007430112157309A0075301121203077
:1001D0009A007630112120309A00773011214F306B
:1001E0009A007830112153309A0079301121433030
:1001F0009A007A30112141309A007B3011214C3025
:100200009A007C30112120309A007D30112120305D
:100210009A007E30112100309A007F301121831224
:1002200008009B001C1555309D00AA309D009C14B1
:060230009C1818290800CB
:02400E00A43FCD
:00000001FF
